:1000000033C2000056C2000054C2000052C20000B9
:1000100050C200004EC200004CC200004AC20000A4
:1000200048C2000046C2000044C200001BC40000D9
:1000300040C200003EC200003CC200003AC20000C4
:1000400096C5000036C2000034C2000032C2000073
:1000500030C200002EC200002CC200002AC20000E4
:1000600028C2000026C200000A000B000C000D0090
:100070000E000F00100011001200130014001500F4
:1000800016001700180019001A001B001C001D00A4
:100090001E001F0020002100220023002400250054
:1000A00026002700280029002A002B002C002D0004
:1000B0002E002F00300031003200330034003500B4
:1000C00036003700380039003A003B003C003D0064
:1000D0003E003F0040004100420043004400450014
:1000E00046004700480049004A004B004C004D00C4
:1000F0004E004F0050005100520053005400550074
:1001000056005700580059005A005B005C005D0023
:100110005E005F00600061006200630064006500D3
:1001200066006700680069006A006B006C006D0083
:100130006E006F0070007100720073007400750033
:1001400076007700780079007A007B007C007D00E3
:100150007E007F0080008100820083008400850093
:1001600086008700880089008A009500A100AC0005
:10017000B800C300CF00DA00E600F100FD0008017E
:1001800014011F012B01360142014D015901640187
:1001900070017B01870192019E01A901B501C00197
:1001A000CC01D701E301EE01FA01050211021C02A4
:1001B000280233023F024A02560261026D027902AE
:1001C000840290029B02A702B202BE02C902D502BB
:1001D000E002EC02F70203030E031A0325033103C6
:1001E0003C03480353035F036A03760381038D03D3
:1001F0009803A403AF03BB03C603D203DD03E903E3
:10020000F40300040B04170422042E0439044504EB
:1002100050045C04680473047F048A049604A104F7
:10022000AD04B804C404CF04DB04E604F204FD0406
:100230000905140520052B05370542054E0559050E
:10024000650570057C05870593059E05AA05B5051E
:10025000C105CC05D805E305EF05FA05060611062C
:100260001D06280601000800080009000A000B000E
:100270000B000C000D000E000E000F00100011000E
:1002800012001200130014001500150016001700CC
:100290001800190019001A001B001C001C001D008A
:1002A0001E001F001F002000210022002300230049
:1002B00024002500260026002700280029002A0007
:1002C0002A002B002C002D002D002E002F003000C6
:1002D0003000310032003300340034003500360085
:1002E00037003700380039003A003B003B003C0043
:1002F0003D003E003E003F00400041004200420001
:1003000043004400450045004600470048004800BF
:1003100049004A004B004C004C004D004E004F007D
:100320004F0050005100520053005300540055003C
:100330005600560057005800590059005A005B00FB
:100340005C005D005D005E005F00600060006100B9
:100350006200630064006400650066006700670077
:10036000680069006A006B0073007C0085008E00E5
:100370009700A000A900B200BB00C400CD00D600C9
:10038000DF00E800F100FA0003010C0114011D0177
:1003900026012F01380141014A0153015C01650129
:1003A0006E0177018001890192019B01A401AD01D9
:1003B000B501BE01C701D001D901E201EB01F40191
:1003C000FD0106020F02180221022A0233023C023A
:1003D00045024E0256025F02680271027A028302EF
:1003E0008C0295029E02A702B002B902C202CB02A1
:1003F000D402DD02E602EF02F70200030903120352
:100400001B0324032D0336033F03480351035A0300
:1004100063036C0375037E03870390039803A103B2
:10042000AA03B303BC03C503CE03D703E003E90368
:10043000F203FB0304040D0416041F042804310412
:10044000390442044B0454045D0466046F047804C8
:1004500081048A0493049C04A504AE04B704C00478
:10046000C904D204DB047F0411241FBECFEFD8E0FF
:10047000DEBFCDBF11E0A0E0B1E0E0E1FDE002C0F1
:1004800005900D92AA31B107D9F721E0AAE1B1E0B8
:1004900001C01D92A73BB207E1F714E0C8E6D4E023
:1004A00003C02297FE012ED4C636D107D1F7CCD295
:1004B000E3C3A6CD259A2D9A22E024BD15BC109247
:1004C0006E00FC01118210820895CF93DF93FC012E
:1004D0008081918186179707A9F19B0140E050E048
:1004E00060E876E988E990E0DDD3C901C92F20E012
:1004F000D22F2097C1F0C830D105C0F0C034D1054B
:1005000058F405C021E001C022E025BD09C023E068
:1005100025BD60E470E004C024E025BD60E071E02A
:10052000ADD367BD0FC061E070E002C068E070E06D
:100530006830710549F36034710549F36130710524
:1005400079F7E0CFDF91CF910895A99B06C0EED255
:1005500087FF02C080E283B9A99A0895EFE6F0E030
:1005600080818D7F80830895F894FB0120E030E046
:1005700061E070E0DC01A20FB31FAB01019002C08B
:10058000440F551F0A94E2F7DF964C932F5F3F4FBD
:100590002830310579F7249A1092800028E02093C2
:1005A00081002091810023602093810020E030E0D1
:1005B0004AB1FC01E20FF31F57AD452B4AB95BB1BD
:1005C00047AD409545234BB92F5F3F4F283031054C
:1005D00079F7FC01E958FF4F2FEF208378940895B5
:1005E0004F925F926F927F929F92AF92BF92CF9203
:1005F000DF92EF92FF920F931F93CF93DF93EC0163
:1006000000E010E087E7E82EF12CEC0EFD1ECC2474
:10061000C394D12C2AE5422E22E6522E22E0622EED
:10062000712CFE01E95BFF4F2081318121153105DD
:10063000B9F05E0187E5A80EB11C40E050E0C301AF
:10064000B20130D3F50131832083C601002E01C0F1
:10065000880F0A94EAF7F7019081982B90830BC0DA
:10066000C601002E01C0880F0A94EAF78095F701B1
:100670009081892380830F5F1F4F229608301105D8
:1006800081F6DF91CF911F910F91FF90EF90DF9056
:10069000CF90BF90AF909F907F906F905F904F9062
:1006A0000895CF93DF939C01FB01C8E0D0E0D9010E
:1006B000A95BBF4F419151916D917C911197641746
:1006C000750719F04D935C93D1E0C1502E5F3F4FF9
:1006D000C111EDCFDD2319F0DF91CF9181CFDF91F3
:1006E000CF910895AF92BF92DF92EF92FF920F9356
:1006F0001F93CF93DF93FC01F0909201A0909301A0
:10070000B0909401DC01A958BF4F0C9110E0DC01BE
:10071000A95ABF4FEF2C80E090E02FEF3FEFD82E8B
:1007200050964D915C9151974A195B0951965C9393
:100730004E935097141615064CF06D917C911197BD
:10074000640F751F51967C936E935097A80102C059
:1007500055954795DA94E2F740FF17C050964D91B2
:100760005C9151974217530730F49F01280F391FAE
:10077000E901EFAC03C04217530739F49F01280F7A
:10078000391FE9012FADE22A9A01019612968830AD
:10079000910529F6E0929201309394012093930100
:1007A0006FB7F89442814431C9F05081852F90E0B1
:1007B0000196DC01AA0FBB1FA80FB91FAE0FBF1F08
:1007C00011963C932E931296FC92852F8F5F843165
:1007D00011F0808301C010824F5F42836FBFDF91B1
:1007E000CF911F910F91FF90EF90DF90BF90AF904E
:1007F0000895CF93DF93EC0102C0CE0173DF8A81AD
:100800008431D9F7DF91CF9108950F931F93CF9340
:10081000DF93EC01EEDF2A812223B1F03981832FAF
:1008200090E00196FC01EE0FFF1FE80FF91FEC0F9F
:10083000FD1F00811181832F8F5F843111F0898327
:1008400001C0198221502A831093890000938800E7
:1008500080916F00826080936F00DF91CF911F9134
:100860000F9108951F920F920FB60F9211242F939C
:100870003F934F935F936F937F938F939F93AF9328
:10088000BF93EF93FF9320911C01222321F130911C
:100890001B01832F90E00196FC01EE0FFF1FE80F74
:1008A000F91FE65EFE4F8081918142813F5F3431C6
:1008B00019F030931B0102C010921B0121502093AC
:1008C0001C018230910508F0019790938900809374
:1008D000880049B903C08AE191E040DEFF91EF91C1
:1008E000BF91AF919F918F917F916F915F914F9148
:1008F0003F912F910F900FBE0F901F90189510925F
:100900001A0110921B0110921C01089510927000A0
:1009100060E071E08AE191E027DE68E071E08AE161
:1009200091E0BFDE8AE191E070DF85EA91E0C2DD0F
:1009300068EE73E085EA91E0C8DD87EA91E0BBC02C
:10094000CF92DF92EF92FF920F931F93CF93DF939B
:1009500087EA91E0BDD085EA91E0F7DD8AE191E098
:1009600048DF60E087EA91E0D8D0F82EF09461E0AB
:1009700087EA91E0D2D0D82ED09462E087EA91E065
:10098000CCD0E82EE0948DEF8E1510F44DEFE42ED0
:1009900085EA91E0DADDC8E0D1E005E911E0C12C9B
:1009A000499159919A01AD2DBC2D9ED129E0969582
:1009B0008795779567952A95D1F733E056954795B2
:1009C0003A95E1F7460F571FF801419351938F0174
:1009D00085EA91E0BADDF1E0C431DF0709F72E2D99
:1009E00030E0220F331FF901E859FF4F85919491B0
:1009F0008093A3019093A4012A593D4FF901859159
:100A000094918093A1019093A20185EA91E09DDDEC
:100A100065E971E08AE191E044DE85EA91E095DDE7
:100A200080E2F89EB0011124625C7F4F85EA91E07C
:100A30004CDD85EA91E0DF91CF911F910F91FF90FE
:100A4000EF90DF90CF9081CDDCD060DF79DFFECFFB
:100A500080E480937C00EAE7F0E080E88083808196
:100A6000876080830895ECE7F0E090819077908331
:100A70009081982B908321E030E0082E01C0220F56
:100A80000A94EAF720937E000895EAE7F0E0808177
:100A900080648083089580917A00829581700895A2
:100AA0002091780030917900932F80E0AC01422BA7
:100AB0009A01C9010895CF93DF93EC01C9DF81E06A
:100AC0008D83D1DFE2DF2098289ADF91CF910895BE
:100AD000CF93DF93EC01DFDF8823B1F0E1DF969560
:100AE0008795969587952D81E22FF0E0EC0FFD1FFD
:100AF000319780832F5F263011F02D8302C081E073
:100B00008D838D81B0DFC1DF189B03C081E08E83B0
:100B100001C01E82DF91CF910895633028F4FC015B
:100B2000E60FF11D8081089580E00895209118015D
:100B300030911901C9019695982F88279795879527
:100B4000822793279C01232F3327269526952695C8
:100B500028273927C901880F991F880F991F8227D5
:100B600093279093190180931801892F08951F925C
:100B70000F920FB60F9211242F933F938F939F9351
:100B8000AF93BF938091AE019091AF01A091B0015E
:100B9000B091B1013091B601232F2D5F2D3720F494
:100BA0000196A11DB11D05C0232F2A570296A11D34
:100BB000B11D2093B6018093AE019093AF01A09335
:100BC000B001B093B1018091B2019091B301A091B5
:100BD000B401B091B5010196A11DB11D8093B20180
:100BE0009093B301A093B401B093B501BF91AF91BD
:100BF0009F918F913F912F910F900FBE0F901F905B
:100C00001895789484B5826084BD84B5816084BD74
:100C100085B5826085BD85B5816085BDEEE6F0E075
:100C2000808181608083E1E8F0E0108280818260D1
:100C30008083808181608083E0E8F0E08081816052
:100C40008083E1EBF0E0808184608083E0EBF0E082
:100C5000808181608083EAE7F0E080818460808326
:100C600080818260808380818160808380818068D0
:100C700080831092C1000895F89448C0AA1BBB1B42
:100C800051E107C0AA1FBB1FA617B70710F0A61B8C
:100C9000B70B881F991F5A95A9F780959095BC01AD
:100CA000CD010895A1E21A2EAA1BBB1BFD010DC0A8
:100CB000AA1FBB1FEE1FFF1FA217B307E407F5070C
:100CC00020F0A21BB30BE40BF50B661F771F881FE8
:100CD000991F1A9469F760957095809590959B017E
:100CE000AC01BD01CF010895A29FB001B39FC00127
:100CF000A39F01D0B29F700D811D1124911D0895F5
:100D0000EE0FFF1F0590F491E02D0994F894FFCFAA
:100D100002030405060700019900B9000B01470111
:0A0D2000D101FF03790125012A002B
:00000001FF
